:030000000219FDE5
:03000B000200AA46
:03002B0002015C73
:03005B000202F9A5
:030073000202E6A0
:1000800002030406080C10182030406080040608A3
:100090000C10182030406080A0C00003070F1F0D17
:1000A0000D04050D050305030302C2AFC0D0C0E077
:1000B000206214E5256009E473E525F4F58AD2622F
:1000C000D0E0D0D0D2AF3285268AC262E526F46075
:1000D0002F30682520720DD0E0D0D0D292D291D2AC
:1000E00090D2AF32D292D291D290206F0C2066097A
:1000F000740AD5E0FDE57B4290D0E0D0D0D2AF329B
:10010000758A00C28DD26201F901B9306805206696
:1001100002C29201B9306805206602C29101B9306D
:100120006805206602C29001B9C29330680A206651
:10013000077408D5E0FDC29201B9C29430680A2064
:1001400066077408D5E0FDC29101B9C29530680A0E
:100150002066077408D5E0FDC29001B9C2AFC2ADF8
:1001600053E6EFC0D0C0E0D2D3D2AFC2CEE52A6012
:1001700007207449152A21BD7800790020742EE5E6
:1001800080307E01F430E40278FF53DACF207E0322
:1001900043DA20307E0343DA10C2D8C271E58030E2
:1001A0007E01F430E40279FFC3E89970CB3061033B
:1001B000752A18207403752A18885CD27020740D73
:1001C000E52B6004152B21CD43DA01C2D820700243
:1001D000413CA85C206102C2702074367982B70469
:1001E00031C3E894F0400374F0F8E8C4540F28F8E1
:1001F0007984B703024112C313C313872120080275
:10020000C313200A06C3C898F8411228F850037493
:10021000FFF88822E52D54066022206B1FE536C3C7
:1002200033C333F8E564C313C313F9C39522400203
:100230008922E82522F52250037522FF7882B60430
:1002400059852224A824C3E52495614002A861C3EE
:10025000E895634002A8638825E5667002418DC376
:10026000E8AA669A5003E8FAE4F9EAC333FBE568C2
:10027000F45B29400D2567F8E56760021567400BC0
:10028000418D0AC3E5679A5002056778FF8826C248
:100290006FC3E52694F84002D26FC3E52594404031
:1002A00002D26420CF0AD0E0D0D043E610D2AD32E3
:1002B000C2CF053A7801E52A6005307402152AC3D9
:1002C000E55C94014005755F0041DC75600075696F
:1002D00000E55F2401F55F5003755FFFD0E0D0D0EB
:1002E00043E610D2AD32C2AF53E67F7592FA7593F2
:1002F000FFC260759104D2AF32C2AF53E6EFC2AD18
:10030000C0D0C0E0C0F0D2D3D2AFA8FBA9FCC2D805
:10031000307102616053DACF207E0343DA10307E01
:100320000343DA20D271E580307E01F420E40261DB
:100330003788278928A18D53DACF207E0343DA201E
:10034000307E0343DA10C2D8C271307402A17978CA
:1003500000E580307E01F430E402A179885CA1617F
:1003600053DACF207E0343DA20307E0343DA10C213
:1003700071206102813953DACF207E0343DA1030D5
:100380007E0343DA20C2D8D27188578958C3E895D2
:1003900055F8E99556F97B007E087A00C3E8948CFD
:1003A000E994005005755B00812B882178A2E6A8AE
:1003B000216055C3E894C8E994005008E4D2E4FBF6
:1003C0007A0A8106C3E89468E994015008E4D2E30C
:1003D000FB7A0F8106C3E894D0E994025008E4D276
:1003E000E2FB7A1E8106C3E894A0E994055008E474
:1003F000D2E1FB7A3C8106C3E89498E9940850085E
:10040000E4D2E0FB7A787E00C3E89559FCE9955A7E
:10041000FD30E70AECF42401FCEDF43400FD755BDB
:1004200000C3EC9AED9E5003755B018859895A858B
:1004300057558558567802A161C3E89527F8E99584
:1004400028F9307C02A145307B02A145307A02A117
:100450003E207502815CE9FDE8FC817BE9C313F96C
:10046000E813F8307902A13EE9C313F9E813F83034
:0F0470007802A13EE9C313FDE813FC20612CC301
:10047F00EC941CED940240028192ED701EC3EC943B
:10048F00C850180529E52970021529C3E529940AD2
:10049F005002A179755C00D270A179E5296002152F
:1004AF00297888E6F97400207F087896B9030278D6
:1004BF009EE624FAFEE43400FFC3EC9EFCED9FFDA4
:1004CF009208B90310A2085007207609D27681E46A
:1004DF00307602C276A2085016B9030DECF424014F
:1004EF00FCEDF43400FD0204FE78007900A145B95B
:1004FF000315EC33FCED33FDC3EC940AFCED9400D3
:10050F00FD50047C007D00C3EC94FFED9400400689
:10051F0078FF7900A145EC8572F0A4C5F0A2F733FE
:10052F00F87900400302056178FF7900020561E95F
:10053F00C313F9E813F8307C0EE9600278FFC3E8C3
:10054F001338F8E43400F9C3E894FFE9940040024B
:10055F0078FF885CD270206102A179741FF4552F47
:10056F004BF52FC274EB7002D274752A18307403D6
:10057F00752A0A306102A18D20740353DAFE2074AC
:10058F0003752B06D0F0D0E0D0D0D2AD43E61032B9
:10059F0079010205BD79030205BD790A0205BD790E
:1005AF001E0205BD79640205BD79C80205BD781725
:1005BF00E4D5E0FDD8FAD9F6227A147B780205E467
:1005CF007A107B8C0205E47A0D7BB40205E47A0B7A
:1005DF007BC80205E47902E4C294D5E0FDC291D54F
:1005EF00E0FDD291D5E0FDD294D5E0FDE920E00207
:1005FF00C29230E002C290E573D5E0FDE920E0023F
:10060F00D29230E002D2907496D5E0FDD9C9EAF8C3
:10061F00D5E0FDD8FBDBBEC29422C37C007D007504
:10062F00F00005F0EA33FAEB33FB50F6EB13FBEA7D
:10063F0013FAC3E9FFE8FEE89AF8E99BF95004EFD3
:10064F00F9EEF8B3EC33FCED33FDD5F0DFEDF9EC5B
:10065F00F822E889F08A20D2D4F8A9F07B0030F78D
:10066F000B7BFFF42401F8E9F43400F9E88520F05E
:10067F00A4ADF0F8E98520F0A4AFF0FEED2EF974EB
:10068F00003FFA7C04C3EA13FAE913F9E813F8DC24
:10069F00F48BF030F70AE8F42401F8E9F43400F9A8
:1006AF00E889F0C2D4F8A9F0227882B604030207D1
:1006BF0013C3E55C940140030206DD852224E4F5B3
:1006CF0044F545F546F547F548C26E0207137882A3
:1006DF00E6FCD26EE522F523783879C7AA40AB4104
:1006EF00C3EB13FBEA13FAEC146013C3EB13FBEA2F
:1006FF0013FAEC14146007C3EB13FBEA13FAD129B6
:10070F008844894522C3E5449523F8E5459400F9CB
:10071F00500CC3E89480E994FF4016020744C3E8E5
:10072F00947FE994005003020744787F7900020711
:10073F0044788079FF8849894A22E5492546F8E5BA
:10074F004A3547F9854A20E4300701F43548FA3035
:10075F00E709C3EA94F04015020782C3EA940F50E9
:10076F000302078278FF79FF7A0F020782780079F8
:10077F00007AF0C3E5249561500AC37401952450A3
:10078F000B0207A0E54A20E70E0207A0E54A30E773
:10079F0006884689478A482278A5E6FAC3E5493391
:1007AF00F8E54A33F9D161E930E70BC3E89480E902
:1007BF0094FF4013E1DAC3E8947FE994005002E11B
:1007CF00DA787F7900E1DA788079FFE820E715C3DE
:1007DF00E52398F84009C3E8940140030208017823
:1007EF0001020801E8F424012523F840030208015F
:1007FF0078FF884B2278A6E6FAA847A94812066127
:10080F00E930E70CC3E89401E994FF40160208367B
:10081F00C3E894FFE99400500302083678FF79008B
:10082F00020836780179FFE920E715C3E54B98F800
:10083F004009C3E89401400302085D780102085D96
:10084F00E8F42401254BF8400302085D78FF882463
:10085F002278FFC26420693D206A12D264C3E54149
:0F086F00940A4009C3E52594405002C26479A160
:10087E00E76023E541601F74FF8541F0848539F000
:10088E00306A0375F005A4F8C5F0600278FFC3E87E
:10089E0095645002A864886322C3E5409440E54104
:1008AE009401E56350031401B8046002F56322025B
:1008BE0008C02275E890227883E6FFE5E820ECF781
:1008CE00A8BDA9BE0570C3E57094084052757000AE
:1008DE00E9FA79A0E76044EA7007E571601B020847
:1008EE00FBC3E895716010E5715006600C140209A7
:1008FE00070460F9020907E571F571C39458401BAE
:10090E007561C0C394044013756180C39404400B99
:10091E00756140C39404400375610075BB0322E505
:10092E00612410500274FFF5617982B704022154DC
:10093E00C3A861E524985002A824C3E89563400239
:10094E00A86388258826E570B4070375BB1022744A
:10095E003279A787F0A4C5F0A2F733F8C3E8956102
:10096E004002A861882288248825882688642275FA
:10097E0040007541F022C2AF75C820A8CCA9CDAAFF
:10098E003A30CF010A75C824D2AFAB3BAC3C883BA2
:10099E00893CC3E89BF8E99C206908F9306702415D
:1009AE009021EDAD3D8A3DF9EA9DFA600478FF791C
:1009BE00FFAE3EAF3F8B3E8C3FA83BA93CC3E89EAB
:1009CE00F8E99FF9C3E54113FBE54013FAE82AF570
:1009DE0040E93BF54150067540FF7541FF4137AA8E
:1009EE0040AB41AC40AD417E047F02C3EB9404406A
:1009FE00021E1FC3EB940840021E1FC3ED13FDEC35
:100A0E0013FCDEF7C3EA9CFAEB9DFBEF6009C3E92A
:100A1E0013F9E813F8DFF7EA28FAEB39FB8A408B73
:100A2E004150067BFF8B408B41C3EB94025002D2A8
:100A3E00673069047F0341627892E6FFC3E537941D
:100A4E008240110FC3E53794A040010FC3EF940607
:100A5E0040027F057E02E541C4540FF9E541C454BE
:100A6E00F0F8E540C4540F28F8C3E89EFAE9940064
:100A7E00FB4009C3EA9402EB940050047A02E4FBB3
:100A8E0041DCAA40AB41EBC4FEEAC4540F4EFCC39A
:100A9E00EA9CFAEB9400FBC3E813C313F8EA28FAB6
:100AAE00EB3400FB8A408B41C3EB94024002C267D9
:100ABE007802EBC4FE7B00EAC4540F4EFAC3EA98E8
:100ACE00FA4005C3940250027A027892E6FF306033
:100ADE000241DC855192855293D26043E680C3E495
:100AEE009AF8E49BF93067026168E8FAE9FBD3E90A
:100AFE0013FDE813FC88518952C3EF94036038EF5D
:100B0E0020E00DE82CF8E93DF9ECFAEDFB020B3193
:100B1E00E828F8E939F9C3E82402F8E93400F97A4B
:100B2E00FE7BFFC3EF9403400E8A538B54884D898E
:100B3E004E8C4F8D50619C885389548A4D8B4E8CB0
:100B4E004F8D503069127553F07554FF754FF07517
:100B5E0050FF7551F07552FF619CE8FAD3E813FC13
:100B6E008851C3EF94036020EF20E007E82CF8ECE7
:100B7E00FA6188E8282402F87AFEC3EF940340084D
:100B8E008A53884D8C4F619C88538A4D8C4FE568F3
:100B9E00C3335002646BF56830600261A67534028F
:100BAE00D26043E680E52D54066034A840A941C3C7
:100BBE00E913F9E813F8C3E913F9E813F8306904F7
:100BCE00E92440F9C2AF53E67F759100C3E498F56E
:100BDE0094E499F595759104D26043E680D2AF22E4
:100BEE00D265754300752000306C03752040020CF1
:100BFE000DD265754300752040306C03752000786A
:100C0E00017901206720E52D54066002C265791432
:100C1E00E541C313700104F8C394144002781430F4
:100C2E006904781B791B206010E543600C30690362
:100C3E00D53404D26D81B071AE0543E59BF45440BA
:100C4E00B52002819A30690908C3E89940011881DC
:100C5E003420650A08C3E8994002810D8134C265CB
:0E0C6E00C2AF53E67F75910030671275940097
:100C7C007595FE759104D26043E680D2AF810DAEBE
:100C8C0040AF41C3E49EF594E49FF595817FC3E5A5
:100C9C003394015002810D306502810DD80281AE72
:100CAC008134C26DC2AF53E67F7591008553948534
:100CBC005495759104854D92854E93D26043E68090
:100CCC00D2AFE52D54066008206A020533020CEC05
:100CDC00306D0D206C0A2065071581158102158673
:100CEC002278003064053065027801E53775F0072D
:100CFC00A4F9E5F028F5F0E9A2F013A2F113A2F2A1
:100D0C0013F537C394785003753778C3E5379538A6
:100D1C004008D266D292D291D290306002A1268540
:100D2C004F92855093D26043E68022D2A0207D164C
:100D3C00C2AF754202C294D293306202C290D2AF5B
:100D4C00759F10020F32C2AF754202C294D2953019
:100D5C006202C292D2AF759F10020F32C2A03072E3
:100D6C0043207D20C2AF75420390013A757B10D2AF
:100D7C0090C295306204C291A188D294D2AF759F73
:100D8C0020020F32C2AF75420390013A757B10D22C
:100D9C0092C293306204C291A1A8D294D2AF759F33
:100DAC0000020F32207D17C2AF754203900115D29D
:100DBC0090306202C291D2AF759F20020F32C2AF47
:100DCC00754203900115D292306202C291D2AF7576
:100DDC009F00020F32D2A0207D16C2AF754204C212
:100DEC0093D295306202C291D2AF759F00020F323E
:100DFC00C2AF754204C295D293306202C291D2AF97
:100E0C00759F20020F32C2A0307243207D20C2AFEA
:100E1C00754205900129757B08D291C29430620409
:100E2C00C292C132D293D2AF759F10020F32C2AFB1
:100E3C0075420590014B757B20D291C294306204AF
:100E4C00C290C152D295D2AF759F10020F32207D45
:100E5C0017C2AF75420590010BD291306202C2925B
:100E6C00D2AF759F10020F32C2AF75420590011FB1
:100E7C00D2913062EBC290D2AF759F10020F32D27A
:100E8C00A0207D16C2AF754206C295D29430620284
:100E9C00C292D2AF759F20020F32C2AF754206C20A
:100EAC0093D294306202C290D2AF759F00020F327F
:100EBC00C2A0307243207D20C2AF75420190014B1D
:100ECC00757B20D292C293306204C290C1DCD29561
:100EDC00D2AF759F00020F32C2AF7542019001294B
:100EEC00757B08D290C295306204C292C1FCD29339
:100EFC00D2AF759F20020F32207D17C2AF75420111
:100F0C0090011FD292306202C290D2AF759F000244
:100F1C000F32C2AF75420190010BD290306202C207
:100F2C0092D2AF759F20C26622900109757B00D2C8
:100F3C0092D291D290C293C294C295C2622278800E
:100F4C0076090876090876040876FF087603087691
:100F5C00FF08760A087603087601087601788C7605
:100F6C00010876FF0876FF0876FF0876FF0876FF03
:100F7C000876030876FF0876FF0876FF08762508C2
:100F8C0076D00876280876500876040876FF08761E
:100F9C000208760008767A0876FF08760108760152
:100FAC00087600087603087600227887E6FFC2727E
:100FBC00BF0302D2727888E6C394036008C27DE650
:100FCC0030E102D27DC27E7889E630E102D27EC366
:100FDC00EF94026008758E01D273020FEE758E00CD
:100FEC00C273227880E6149000809378A5F67881FD
:100FFC00E6149000809378A6F67886E61490008D1F
:10100C009378A7F67886E6F539C3940250037539C0
:10101C0002789CE67538FFB402037538A0B403035C
:10102C0075388278A3E61490009A93F566120F3502
:10103C0022227896E6FA7897E6FB7888E6B40305E0
:10104C00C3EB940EFB307F047A007BFFC3EB9AFC5E
:10105C00C3948250027C827572000572EC8572F02A
:0D106C00A4C3E5F0947D40F222D27F113E36
:101079001205AE7A007B007C101205A4E55C2AFA01
:1010890074003BFBDCF37C04C3EB13FBEA13FADCCF
:10109900F7FEC27F113E22E5EF20E6037520000529
:1010A90020903FFFE520146006901DFF1460009317
:1010B90004600375EF1253D9BF7581C043FF8012D5
:1010C900059F75EF0243B203E5B3240220E70DF54E
:1010D90021E5E320E0068521B343E301120F3575CD
:1010E90080FF75A40075F1D475D4EF75908775A547
:1010F9004075F2FF75D5BF75A60175E24275DB46ED
:1011090075EA02120F35E4F8F6D8FD756801120F79
:101119004A1215D778988673753001C2AF1205B88F
:101129001205C81205AE1205CF1205AE1205D61268
:1011390005AEC2AF78FA79FA308407D9FBD8F7023D
:101149001C00120FB6120FEF113D113E78988673ED
:10115900120F3575881075890275C8247591047543
:10116900D84075A82275B80275E690759B80759D63
:101179000075D10E75BC5875BB0375BA1175E88039
:1011890012059FD2AF1208BD75360053DACF207E03
:101199000343DA20307E0343DA1043DA01C2D8C2AE
:1011A900711205B8D2617B037A0CE55B70077A0C82
:1011B900DB0302113B1205AE20700302113BC27022
:1011C900E55CC3940240E1E52F541F855E5DF55E41
:1011D900B55DD5DAD5C26153DACF207E0343DA2073
:1011E900307E0343DA10C2D8C27178A2E67008D201
:1011F90074E52F54E0F52FC2757529001205B33037
:101209007409C3E529940A4002D2751205A478022B
:101219003074027800C3E55C9840F0C2AF1205C88B
:101229001205C81205C8D2AF1205B8754C007888E6
:10123900E6B4030261131205A4788CE6C394015045
:1012490003021313E530C3940150030213132074EE
:1012590035C3E55C94FF5003021313C2AF1205DDD9
:10126900D2AF1205B3C3E55C940150EFC2AF1205CA
:10127900C81205A91205C8D2AF1205B3C3E55C941B
:10128900FF40E902177F7F02D27F113E1205B3C2E8
:10129900AFC27F113EAE5CC3E55C947FD2AF4074B0
:1012A90012059FC2AF1205DDD2AFDFDC1175C3EEA7
:1012B9007897F61205B81216191217027F0AD27F0B
:1012C900113E1205B3C2AFC27F113EAE5CC3E55CED
:1012D900947FD2AF50E612059FC2AF1205C812051E
:1012E900A91205C8D2AFDFD61175EE24037896F698
:1012F9001205B81216191217311205B3113EC3E5BA
:101309005C94FF5002415702177FC3E55C954C403E
:1013190003855C4C1205B378017988E7B403027838
:1013290005C3E55C9840024137C2AF1205DD1205DD
:10133900DD1205DDD2AF1205B8753000E4F531F5DF
:10134900320531E531F4703F0532789AE67819149F
:101359006012783214600D787D14600878FA146090
:1013690003753200C3E53298401D120F3512059FEF
:10137900153275310078998673C2AF1205DDD2AF87
:10138900789886731205B31205A9E52A7005307499
:1013990002213B78012074027806C3E55C9840A1DC
:1013A9007888E6C3940360031205B3E52A70030243
:1013B900113BC2AF120F35E4F522F523F524F525CB
:1013C900F526F567D2AF7885E6C333F565E4F544CC
:1013D900F545F546F547F548F570F52CF52DF53742
:1013E90075700875BB1012059F1208C1E5E820EC5D
:1013F900FBA8BDA9BEE97001F888711208C575700E
:101409000875BB10120FB6C2AF7561FF12095D8571
:101419002261852262852263D2AF7522017524017A
:10142900752501752601856069756A017888E6B4B4
:101439000307C27D307602D27DD268D26975330046
:10144900120E8B120EBC12097D12098412097D122B
:10145900098412097D120BFF1206B8120CED120D48
:0D14690037120984120BEE306E03120714C7
:101476002067031208603067031208A7120CED12EA
:101486000D68120984120BFF306E03120749120C05
:10149600ED120DE1120984120BEE306E031207A74E
:1014A600120CED120E12120984120BFF306E03128B
:1014B6000804120CED120E8B1209841208C1120BCD
:1014C600EE120CED120EBC1208C5120984306932F8
:1014D600856461856462856069756A0179187A0C2C
:1014E600C3E53399400FC269D26A8A35856461853E
:1014F6006463021508C3E55C9401400302145E02AE
:10150600158E306A1D206C1AE535147006C26AD233
:101516006B815EF535C3E55C9401400302145E02FF
:10152600158E75360078FA79A4E760027803C3E56C
:101536005F985054307404E52A604D7888E6B40309
:1015460017207D05207607A15E307602A15E206C0D
:1015560007D26C856461819D78F0306C0585646185
:101566007820C3E541985002815E306C1BC26CC284
:101576007D307602D27DD26A753512856461815ED0
:101586000536E55C6002A191753600C2AF120F35D3
:101596007887E6FE7602120FB67887EEF6E4F52235
:1015A600F523F524F525F526F565752C00752D0032
:1015B600D2AF1205B3120F3578A4E66006C292C206
:1015C60091C290307409C3E53694044002213B6110
:1015D60045901A0D782012165BE520B4550CA3121F
:1015E600165BE520B4AA030215F9120F4A12161962
:1015F600021618901A0378807B0A12165BA308DB82
:10160600F9901A0F788C7B1912165BA308DBF990F8
:101616001A2822C2AF12169A121674901A00740E65
:10162600121660A37406121660A374151216609043
:101636001A0378807B0A12165FA308DBF9901A0F4B
:10164600788C7B1912165FA308DBF91216AD1216F9
:101656008B901A2822E493F622E6438F01538FFDDE
:1016660075EF0275B7A575B7F1F0538FFE22438F5C
:1016760002438F0175EF0275B7A575B7F1901A0D84
:10168600F0538FFC22901A0D7455D160901A0E7487
:10169600AAD160227A3079D07820901A40D15BE5C1
:1016A60020F709A3DAF7227A3079D0901A40E7D1E9
:1016B6006009A3DAF922AB74A875BB01027980BB75
:1016C60002027981BB03027982BB04027984BB05DD
:1016D600027986BB06027992BB07027987BB0802AC
:1016E60079A3BB0902799CBB0A027988BB0B0279F4
:1016F60089E8F7227C051205B8DCFB22C2AF120589
:10170600C81205CF1205D61205DD1205A91205C8A5
:101716001205CF1205D61205DD1205A91205C8124B
:1017260005CF1205D61205DDD2AF22C2AF1205DDF6
:101736001205D61205CF1205C81205A91205DD122B
:1017460005D61205CF1205C81205A91205DD120528
:10175600D61205CF1205C8D2AF22AE74AF75C2AF8E
:101766001205C81205C81205C81205A9DEF212052F
:10177600DD1205A9DFF8D2AF22F102D1FAD1FA754E
:101786007401757501757600F1607C05AD5C120516
:10179600B8C3ED955C70F5C3E55C9401400AC3E5FA
:1017A6005C94FF40320217BBD1BCD119F102C2AF23
:1017B60075EF12D1FADCD50576C3E57694035002AF
:1017C60080C6D1FA0575E5741490009F93F808C396
:1017D600E57598500280AED1FAD1FA0574C3E57466
:1017E600940C5002809C120F4AD119C2AF75EF12A9
:0217F600D1FA26
:0319FD000210A035
:101A00000E0615090904FF03FF0A03010155AA0187
:101A1000FFFFFFFFFF03FFFFFF25D0285004FF0259
:091A2000007AFF0101000300FF40
:101A400023484B696E67323041232020202020201C
:101A500023424C48454C4923463333302320202031
:101A60002020202020202020202020202020202076
:101C0000C2AFC2D353D9BF7581C043B20343FF8073
:101C1000752438752503B1C975EF0275E24043F1AB
:101C20001053A4EF75D4FFD2847DFA780379E67C53
:101C300010752200752300901DD67B0675249875BB
:101C400025013084028142208408D8FBD9F9DCF7D1
:101C500081B4308408D8FBD9F9DCF781B4B189E4C8
:101C600093A3C39A6004DDC381B4DBDBB17B600264
:101C7000812B7B08E493FAA3B15CDBF87A30B15C8A
:101C8000752200752300B17BEAFCEBFDC3ED94FEE9
:101C9000400EB17B8A278B28ED30E0048A828B834B
:101CA000B17B7AC270D8C3ED94FE601350CEBD00F4
:101CB00025EC60097520007521FF0200008100A855
:101CC00027A9280809D804D90281D3B17FEA89AAB3
:101CD000F281C50D81A0C3ED94035049EDA2E092BD
:101CE000007AC5C3E5829400E583941C50902000DF
:101CF00010438F02438F0175B7A575B7F1F030001F
:101D00001FA827A9280809438F01538FFDD804D99C
:101D100002A12089AAE275B7A575B7F1F0A3A10DBC
:101D2000538FFC817C7AC1BD030CE493A3FAB140CC
:101D3000DCF8B138817C817EAA22AB23B15CEBFA5E
:101D4000EA6222752608C3E52313F523E52213F57D
:101D50002250066323A0632201D526EAB1C9B1C986
:101D600075260AEAF4200102D284300102C284B14D
:101D7000C9C3134002C201D526EB22B17FEAFB2082
:101D80008402A17F308402A184752608AE24AF2589
:101D9000C3EF13FFEE13FEB1CDB1C9C3EA13308414
:101DA000024480FA30E703632201C3E52313F523DD
:101DB000E52213F52250066323A0632201D526D91C
:101DC000E52265236523F52222AE24AF250E0FDE22
:101DD000FEDFFCD20122424C48656C693437316326
:041DE000F3300601D5
:00000001FF
